:020000040000FA
:02000000762860
:0800080076288C0081018316AB
:100010000313C030810508008C008101831603138F
:10002000C030810501308104831203130B110B1DB5
:1000300017288C0B162808008E00E13086050E0D5F
:100040001E39860408009214262892108F003A2048
:10005000921C86170F080F0E1C2036200F081C203C
:100060003620E13086058613061308008616000048
:100070008612080086131214831603131E3086049A
:100080008312031306178616061E1210861200002E
:10009000362012184328061383160313E130860511
:1000A00083120313080017141508980008309300F2
:1000B0003030981B31302520980D930B5828171C91
:1000C0000800171016085528990008309400991F49
:1000D0000511991B0515990D0000851500001910D3
:1000E000051A19148511940B672808008316031349
:1000F0000130860583120313861206138613E1303E
:10010000860504300C2003301C20362001300C20E2
:1001100008301C20362001300C2002301C203620F4
:1001200001300C20283023200C30232028302320BD
:100130000130232083160313F0308500831203134C
:10014000033085004E3025205330252043302520B4
:1001500020302520413025204430252043302520E3
:1001600031302520323025203130252033302520F4
:1001700030302520203025204330252049302520CF
:100180004E302520C03023205430252065302520D6
:1001900073302520743025202D302520493025202E
:1001A0006E302520743025206530252072302520C2
:1001B00066302520613025206330252065302520DC
:1001C0001030052007301320FC30850530306420C6
:1001D000033085040130232053302520743025203E
:1001E000613025207430252075302520733025207E
:1001F000FC30850534306420190895008515000011
:100200009601051A9617851103308504873023203F
:1002100053201930052007301320FC308505F830B5
:1002200064200330850401300C20FC30850520302B
:1002300064200330850403300C20FC308505243015
:1002400064200330850401300C20FC3085053030FB
:1002500064200330850401300C20FC308505843097
:10026000642019089500851500009601051A961757
:1002700085110330850487302320532001300C2062
:10028000FC30850584306420190895008514003001
:1002900064201908960003308504C03023205320C1
:0202A0003E29F5
:02400E00F13F80
:00000001FF
